S0220000687474703A2F2F737265636F72642E736F75726365666F7267652E6E65742F1D
S12300000C9438000C9454270C94AA1F0C945F000C945F000C945F000C94A81E0C945F001E
S12300200C945F000C948C290C945F000C94482D0C945F000C94DA200C94B4200C94F61E93
S12300400C94092E0C945F000C942E2E0C945F000C94C32E0C948B2E0C945F000C945F00E3
S12300600C945F000C945F000C945F000C945F0011241FBECFEFD0E1DEBFCDBF14BEA895C7
S123008088E10FB6F89480936000109260000FBE13E0A0E0B1E0E4E2F1E602C005900D92C9
S12300A0A23FB107D9F718E0A2EFB3E001C01D92A939B107E1F70E9433170C9490300C94E9
S12300C000009C01F999FECF32BD21BDF89A80B508959C01F999FECF1FBA32BD21BD60BD30
S12300E00FB6F894FA9AF99A0FBE089520E030E0F999FECF28593D4F32BD21BD28563240E1
S1230100F89A80B5F901EE59F94F80832F5F3F4F81E02034380761F720E030E0F999FECFB1
S123012028573E4F32BD21BD28583140F89A80B5F901E25CFE4F80832F5F3F4F25303105FB
S123014069F712BC11BC089580E090E0FC01EE59F94FE081F999FECF1FBA88599D4F92BDF2
S123016081BDE0BD0FB6F894FA9AF99A0FBE8756924021E08034920749F712BC11BC0895E6
S123018020E030E0F999FECF205F3F4F32BD21BD20513040F89A80B5F901ED52FB4F8083E4
S12301A02F5F3F4F81E02034380761F712BC11BC089580E090E0FC01ED52FB4FE081F99952
S12301C0FECF1FBA409692BD81BDE0BD0FB6F894FA9AF99A0FBE0F9721E08034920759F7EC
S12301E012BC11BC089520E430E0F999FECF205B3E4F32BD21BD20553140F89A80B5F901D4
S1230200EB5BFE4F80832F5F3F4F203A310569F712BC11BC089580E490E0FC01EB5BFE4F9C
S1230220E081F999FECF1FBA805B9E4F92BD81BDE0BD0FB6F894FA9AF99A0FBE8F54914036
S1230240803A910551F712BC11BC0895F999FECF82E090E092BD81BDF89A80B590E09093B2
S1230260200180931F0140911F0150912001F999FECF83E090E092BD81BDF89A20B5922F4C
S123028080E0840F951F9093200180931F01F999FECF8DEE93E092BD81BDF89A80B590E02B
S12302A090932401809323014091230150912401F999FECF8EEE93E092BD81BDF89A20B57E
S12302C0922F80E0840F951F909324018093230180911F0190912001909322018093210145
S12302E0F999FECF84E090E092BD81BDF89A80B590E09093260180932501409125015091A8
S12303002601F999FECF85E090E092BD81BDF89A20B5922F80E0840F951F909326018093C5
S12303202501F999FECF86E090E092BD81BDF89A80B590E09093010180930001409100018F
S123034050910101F999FECF87E090E092BD81BDF89A20B5922F80E0840F951F90930101FF
S123036080930001F999FECF81E090E092BD81BDF89A80B58093F203F999FECF88E090E0A2
S123038092BD81BDF89A80B580931301F999FECF89E591E092BD81BDF89A80B580932F0109
S12303A0F999FECF82E094E092BD81BDF89A90B5892F8150883078F080912F01843039F4D5
S12303C081E08093180183E68093180606C082E08093180102C090931801F999FECF89E0D8
S12303E090E092BD81BDF89A80B580931201F999FECF84E094E092BD81BDF89A80B5809371
S1230400BF048091BF04823E14F482EE05C08091BF048F311CF08EE18093BF04F999FECF00
S12304208EE090E092BD81BDF89A80B580932801F999FECF8BE090E092BD81BDF89A80B5BC
S123044020911801829FC001112490931A0180931901F999FECF83E094E092BD81BDF89AF7
S123046080B580931B01F999FECF8CE090E092BD81BDF89A80B520911801829FC0011124A4
S123048090931D0180931C01F999FECF8FE691E092BD81BDF89A80B580931E01F999FECFBD
S12304A082EF91E092BD81BDF89A80B58093670480916704882319F081E080936704F999E3
S12304C0FECF8DE090E092BD81BDF89A80B526E0829FC00111249093150180931401F9990A
S12304E0FECF81E791E092BD81BDF89A80B580933C06F999FECF80E791E092BD81BDF89A53
S123050080B580933A068AE08093CB0781E08093C907F999FECF8FE891E092BD81BDF89A56
S123052080B5809330018091300181FF05C080913001827F809330018091300185FF05C0A5
S1230540809130018F7280933001F999FECF84EF91E092BD81BDF89A80B590E02CE231E0EA
S1230560AC01429FC001439F900D529F900D11249093CF048093CE04F999FECF85EF91E0C7
S123058092BD81BDF89A80B58093CB04F999FECF86EF91E092BD81BDF89A80B58093C904A8
S12305A0F999FECF87EF91E092BD81BDF89A80B58093C804F999FECF88EF91E092BD81BDEA
S12305C0F89A80B590E09093C7048093C6044091C6045091C704F999FECF89EF91E092BD37
S12305E081BDF89A20B5922F80E0840F951F9093C7048093C604F999FECF8BEF91E092BD86
S123060081BDF89A80B590E090933201809331014091310150913201F999FECF8CEF91E064
S123062092BD81BDF89A20B5922F80E0840F951F9093320180933101F999FECF8DEF91E073
S123064092BD81BDF89A80B590E090933401809333014091330150913401F999FECF8EEF3C
S123066091E092BD81BDF89A20B5922F80E0840F951F9093340180933301F999FECF8FEF2D
S123068091E092BD81BDF89A80B590E090937803809377034091770350917803F999FECFF0
S12306A080E092E092BD81BDF89A20B5922F80E0840F951F9093780380937703F999FECF7E
S12306C08BEC93E092BD81BDF89A80B580937F04F999FECF8CEC93E092BD81BDF89A80B5A4
S12306E090E09093810480938004F999FECF8DEC93E092BD81BDF89A80B580938904F99976
S1230700FECF8EEC93E092BD81BDF89A80B58093790320E030E0F999FECF225A3E4F32BDD1
S123072021BD2E553140F89A80B5F901EB51FE4F8083F999FECF2E583E4F32BD21BD2257DE
S12307403140F89A80B5F901E75EF94F8083F999FECF24583E4F32BD21BD2C573140F89A18
S123076080B5F901E75EF94F808B2F5F3F4F2A30310509F0D0CFF999FECF87E092E092BDE3
S123078081BDF89A80B580933901F999FECF83E092E092BD81BDF89A80B580933A0120E02D
S12307A030E094E6F901E855F84F908BF999FECF245E3D4F32BD21BD2C513240F89A80B522
S12307C0F901E855F84F80832F5F3F4F2031310549F720E030E0F999FECF27593E4F32BD46
S12307E021BD29563140F89A80B5F901E65DFE4F80832F5F3F4F2430310569F720E030E0BD
S1230800F999FECF225D3D4F32BD21BD2E523240F89A80B5F901E454FC4F80832F5F3F4F48
S12308202031310569F7F999FECF8DE691E092BD81BDF89A80B580932701F999FECF81EF2C
S123084091E092BD81BDF89A80B580936604F999FECF80EF91E092BD81BDF89A80B58093AC
S12308602E01F999FECF86E092E092BD81BDF89A80B58093290120E030E0F999FECF2A5490
S12308803C4F32BD21BD265B3340F89A80B5F901E151FE4F80832F5F3F4F2031310569F7C2
S12308A0F999FECF87EC93E092BD81BDF89A80B580933C01F999FECF88EC93E092BD81BD78
S12308C0F89A80B580933D01F999FECF84ED93E092BD81BDF89A80B580937204F999FECF7D
S12308E085ED93E092BD81BDF89A80B580937304F999FECF86ED93E092BD81BDF89A80B598
S123090080937404F999FECF87ED93E092BD81BDF89A80B580937504F999FECF88ED93E0DB
S123092092BD81BDF89A80B580937604F999FECF89ED93E092BD81BDF89A80B580937704A8
S1230940F999FECF8AED93E092BD81BDF89A80B580937804F999FECF8BED93E092BD81BD90
S1230960F89A80B580937904F999FECF88EE93E092BD81BDF89A80B590E0909336018093A3
S123098035014091350150913601F999FECF89EE93E092BD81BDF89A20B5922F80E0840F0D
S12309A0951F9093360180933501F999FECF8AEE93E092BD81BDF89A80B580936904F9992C
S12309C0FECF8CEC93E092BD81BDF89A80B52AE0829FC00111249093810480938004F99915
S12309E0FECF81ED93E092BD81BDF89A80B52AE0829FC00111249093860480938504F999F5
S1230A00FECF82ED93E092BD81BDF89A80B52AE0829FC0011124909388048093870412BC93
S1230A2011BC089520911F0130912001F999FECF1FBA82E090E092BD81BD20BD0FB6F894D0
S1230A40FA9AF99A0FBE20911F0130912001F999FECF1FBA83E090E092BD81BD30BD0FB6A1
S1230A60F894FA9AF99A0FBE2091250130912601F999FECF1FBA84E090E092BD81BD20BDBD
S1230A800FB6F894FA9AF99A0FBE2091250130912601F999FECF1FBA85E090E092BD81BDB4
S1230AA030BD0FB6F894FA9AF99A0FBE2091000130910101F999FECF1FBA86E090E092BD2E
S1230AC081BD20BD0FB6F894FA9AF99A0FBE2091000130910101F999FECF1FBA87E090E02E
S1230AE092BD81BD30BD0FB6F894FA9AF99A0FBE20911301F999FECF1FBA88E090E092BD0F
S1230B0081BD20BD0FB6F894FA9AF99A0FBE20911201F999FECF1FBA89E090E092BD81BD0F
S1230B2020BD0FB6F894FA9AF99A0FBE12BC11BC0895F999FECF1FBA81EF91E092BD81BDB1
S1230B4010BC0FB6F894FA9AF99A0FBEF999FECF1FBA80EF91E092BD81BD8AE080BD0FB66F
S1230B60F894FA9AF99A0FBE20916704F999FECF1FBA82EF91E092BD81BD20BD0FB6F89400
S1230B80FA9AF99A0FBEF999FECF1FBA89E591E092BD81BD84E080BD0FB6F894FA9AF99AA0
S1230BA00FBEF999FECF1FBA81E092E092BD81BD87E180BD0FB6F894FA9AF99A0FBEF99950
S1230BC0FECF1FBA82E092E092BD81BD8EE180BD0FB6F894FA9AF99A0FBEF999FECF1FBAE1
S1230BE08CE090E092BD81BD85E080BD0FB6F894FA9AF99A0FBEF999FECF1FBA8FE691E083
S1230C0092BD81BD82E380BD0FB6F894FA9AF99A0FBEF999FECF1FBA81E791E092BD81BDBE
S1230C2084E180BD0FB6F894FA9AF99A0FBEF999FECF1FBA80E791E092BD81BD81E080BD8E
S1230C400FB6F894FA9AF99A0FBEF999FECF1FBA84EF91E092BD81BD88EC80BD0FB6F894A0
S1230C60FA9AF99A0FBEF999FECF1FBA85EF91E092BD81BD81E080BD0FB6F894FA9AF99ABC
S1230C800FBEF999FECF1FBA86EF91E092BD81BD84E180BD0FB6F894FA9AF99A0FBEF9995F
S1230CA0FECF1FBA87EF91E092BD81BD8AE580BD0FB6F894FA9AF99A0FBEF999FECF1FBAED
S1230CC088EF91E092BD81BD88EE80BD0FB6F894FA9AF99A0FBEF999FECF1FBA89EF91E082
S1230CE092BD81BD83E080BD0FB6F894FA9AF99A0FBE2091310130913201F999FECF1FBA6F
S1230D008BEF91E092BD81BD20BD0FB6F894FA9AF99A0FBE2091310130913201F999FECFFF
S1230D201FBA8CEF91E092BD81BD30BD0FB6F894FA9AF99A0FBE2091330130913401F999BE
S1230D40FECF1FBA8DEF91E092BD81BD20BD0FB6F894FA9AF99A0FBE209133013091340172
S1230D60F999FECF1FBA8EEF91E092BD81BD30BD0FB6F894FA9AF99A0FBE2091770330919E
S1230D807803F999FECF1FBA8FEF91E092BD81BD20BD0FB6F894FA9AF99A0FBE20917703D3
S1230DA030917803F999FECF1FBA80E092E092BD81BD30BD0FB6F894FA9AF99A0FBEF99998
S1230DC0FECF1FBA87E092E092BD81BD8CED80BD0FB6F894FA9AF99A0FBEF999FECF1FBAD0
S1230DE083E092E092BD81BD86EE80BD0FB6F894FA9AF99A0FBE8CE192E028ECF999FECF45
S1230E001FBA92BD81BD20BD0FB6F894FA9AF99A0FBE019632E08C32930781F7F999FECF6E
S1230E201FBA8FE891E092BD81BD82E280BD0FB6F894FA9AF99A0FBEF999FECF1FBA86E0DC
S1230E4092E092BD81BD81E080BD0FB6F894FA9AF99A0FBE12BC11BC08958F929F92AF92E1
S1230E60BF92CF92DF92EF92FF920F931F93CF93DF93C0E0D0E035E0832E32E0932E23ED18
S1230E80A22E23E0B22EF999FECF92BC81BCF89A60B5F999FECFB2BCA1BCF89AE0B46E014B
S1230EA0CC0CDD1C2FEF31E0C20ED31EF6012081318170E080E090E040E050E00E940130E0
S1230EC0FF2400E010E0A80197010E94013024E630E040E050E00E94533079018A01C801AA
S1230EE0B70124EF31E040E050E00E94013028EC30E040E050E0E20EF31E041F151FA8017A
S1230F0097010E945330CA01B9012FEF30E040E050E00E94013025E030E040E050E00E9433
S1230F20533082E0220F331F441F551F8A95D1F7CA01B90124E630E040E050E00E94533073
S1230F40F601318320832196C732D10509F09BCFC0E0D0E009EC802E03E0902E13EDA12EF3
S1230F6013E0B12EF999FECF92BC81BCF89A60B5F999FECFB2BCA1BCF89AE0B46E01CC0C73
S1230F80DD1C2DE432E0C20ED31EF6012081318170E080E090E040E050E00E940130FF24C0
S1230FA000E010E0A80197010E94013024E630E040E050E00E94533079018A01C801B70134
S1230FC024EF31E040E050E00E94013028EC30E040E050E0E20EF31E041F151FA8019701B9
S1230FE00E945330CA01B9012FEF30E040E050E00E94013025E030E040E050E00E94533068
S1231000A2E0220F331F441F551FAA95D1F7CA01B90124E630E040E050E00E945330F601DE
S1231020318320832196C732D10509F09BCFC0E0D0E0FAEC8F2EF3E09F2EE3EDAE2EE3E06A
S1231040BE2EF999FECF92BC81BCF89A60B5F999FECFB2BCA1BCF89AE0B46E01CC0CDD1C7F
S12310602BE932E0C20ED31EF6012081318170E080E090E040E050E00E940130FF2400E0F5
S123108010E0A80197010E94013024E630E040E050E00E94533079018A01C801B70124EF20
S12310A031E040E050E00E94013028EC30E040E050E0E20EF31E041F151FA80197010E9449
S12310C05330CA01B9012FEF30E040E050E00E94013025E030E040E050E00E94533062E0E7
S12310E0220F331F441F551F6A95D1F7CA01B90124E630E040E050E00E945330F60131830C
S123110020832196C732D10509F09BCFC0E0D0E034E0832E32E0932E23EDA22E23E0B22E94
S1231120F999FECF92BC81BCF89A60B5F999FECFB2BCA1BCF89AE0B46E01CC0CDD1C29EE73
S123114032E0C20ED31EF6012081318170E080E090E040E050E00E940130FF2400E010E038
S1231160A80197010E94013024E630E040E050E00E94533079018A01C801B70124EF31E01E
S123118040E050E00E94013028EC30E040E050E0E20EF31E041F151FA80197010E945330F6
S12311A0CA01B9012FEF30E040E050E00E94013025E030E040E050E00E94533082E0220F38
S12311C0331F441F551F8A95D1F7CA01B90124E630E040E050E00E945330F6013183208399
S12311E02196C732D10509F09BCFDF91CF911F910F91FF90EF90DF90CF90BF90AF909F9049
S12312008F900895EAE7F0E0108210927C0080E880BF87EE808311B885E090E090930104D8
S12312208093000488E790E09093F5038093F40384E690E0909303048093020490930B0440
S123124080930A0486E490E0909305048093040408950F931F93CF93DF93282F30E0F90122
S1231260EE0FFF1FEE5FFE4F0081118183E0033F180718F0E2E3F0E04AC083E00F3D180769
S123128018F0EAE0F0E043C0A0E0B0E087E290E0289FA001299F500D389F500D1124EA01DB
S12312A0CA0FDB1FCC0FDD1FC150DE4F888199818017910730F5FD013197E40FF51FEE0F01
S12312C0FF1FE150FE4F208131816081718148815981FD01EE0FFF1FEE0FFF1FEA0FFB1F5E
S12312E03596201B310BC901880F991F880F991F641B750B820F931F0E942C30E60FF71FF5
S123130006C01196A732B10551F6E8ECF0E0CF01DF91CF911F910F9108950F931F93CF939F
S1231320DF93AC01E0E0F0E0EF01CC0FDD1FDE01A95CBC4F8D919C91119748175907C0F5DD
S12313406D917C913197EE0FFF1FDF01A95CBC4F8D919C911197681B790B8D919C91C15B4A
S1231360DC4F28813981E15BFC4F00811181481B590B84E690E0DC014A9FC0014B9F900D92
S12313805A9F900D11240E942C30201B310B0190F081E02D629FC001639F900D729F900DEB
S12313A0112464E670E00E942C306E0F7F1F09C03196EA30F10509F0B7CF609163037091CA
S12313C06403CB01DF91CF911F910F9108958091F4039091F503282F205527FF0AC080912B
S12313E01401909115019C01220F331F280F391F1FC02F312CF0209114013091150118C01E
S12314004091140150911501332727FD309588E290E0821B930B9C01249FC001259F900D11
S1231420349F900D11246AE070E00E942C309B01C90108950F931F93CF93DF93AC01809182
S12314407A0390917B034817590718F4E0EFF0E057C080919603909197038417950718F443
S1231460E0E0F0E04DC0E1E0F0E0EF01CC0FDD1FDE01A658BC4F8D919C91119748175907D9
S1231480C0F56D917C913197EE0FFF1FDF01A658BC4F8D919C911197681B790B8D919C9177
S12314A0E856FC4F20813181C856DC4F08811981481B590B84E690E0DC014A9FC0014B9FCE
S12314C0900D5A9F900D11240E942C30201B310B0190F081E02D629FC001639F900D729FAA
S12314E0900D112464E670E00E942C30E61BF70B07C03196EE30F10509F0B7CFEEEFF0E0AD
S1231500CF01DF91CF911F910F91089580917E04882359F08CED95E090933801809337011E
S123152010929804109297042AC080917E04882349F08CED95E0909338018093370184E6CC
S123154090E019C080917E04882349F08CED95E090933801809337018AEF90E00CC080916C
S12315607E04882361F08CED95E0909338018093370184EF91E09093980480939704F89477
S123158080916204909163048A5A9A4AC1F080916204909163048555954589F07894809186
S12315A0A3079091A40780649093A4078093A30784EF91E090933801809337010AC07894E1
S12315C08091A3079091A4078F7B9093A4078093A307F89480916404909165048F3F89F015
S12315E078948091A3079091A40780689093A4078093A30784EF91E0909338018093370156
S12316000AC078948091A3079091A4078F779093A4078093A3078091370190913801892B81
S1231620B1F15E9A20919704309198042115310511F45E9A19C08091950490919604029723
S123164098F48BB18295869586958370809581708295880F880F807C9BB19F7B982B9BB9BA
S12316603093960420939504809195049091960401979093960480939504809137019091ED
S123168038010197909338018093370108955E98109298041092970408958091A307909147
S12316A0A4079F779093A4078093A307809100019091010197FD44C08091F20380FF32C096
S12316C02091590430915A0480912101909122018C599F4F8217930720F441E050E060E8AF
S12316E032C02091590430915A04809121019091220149978217930720F441E050E068E090
S123170022C02091590430915A048091210190912201845690408217930790F441E050E08D
S123172064E011C02091590430915A0480912101909122018217930718F440E050E802C093
S123174040E050E060E02091A3073091A407CA019927869597958827822B932B9093A40774
S12317608093A3072091A3073091A407CA0180709078822B932B9093A4078093A307809117
S123178000019091010192FF32C02091590430915A0480913101909132018217930738F57A
S12317A02091590430915A04809133019091340128173907E0F4809127012091000430915B
S12317C0010490E08217930794F08091A3079091A40794609093A4078093A3078091F203CD
S12317E080FF03C0416068600BC0506809C08091A3079091A4079B7F9093A4078093A307C2
S1231800209102043091030480913A0190E08217930734F480913A01882311F040616860CD
S123182080917304209104043091050490E08F5B9F4F8217930774F480917304882351F042
S123184040628091590490915A04895B9B40A0F0646012C080917304209104043091050405
S123186090E0C296821793073CF480917304882319F0406271E001C070E0809172042091C1
S12318800A0430910B0490E0C296821793076CF480917204882349F040648091590490916D
S12318A05A04855C994008F06460772321F082E38093550402C010925504309906C040FD4B
S12318C002C057FF09C04170507850937C0440937B0460937D0406C010927C0410927B0478
S12318E010927D0460937E040895809100019091010193FF6EC1339906C0809184048F5FA0
S12319008093840402C01092840480918404853108F454C010927F042091590430915A048B
S123192080917703909178038217930778F480917B0490917C04826090937C0480937B0495
S123194080917D04886080937D0409C080917B0490917C048D7F90937C0480937B04809129
S1231960F20383FF16C08091590490915A04855C994078F080917B0490917C0484609093CF
S12319807C0480937B0480917D04826080937D0409C080917B0490917C048B7F90937C0482
S12319A080937B048091800490918104909383048093820484E3809384048EC0809182042C
S12319C090918304892B09F45CC080918204909183040197909383048093820480917F04E0
S12319E0823099F0833030F4882351F0813009F073C019C08330A9F1843009F06DC031C017
S1231A00109283041092820467C080917B0490917C04846090937C0480937B0480917D046E
S1231A20826080937D042091590430915A0480917703909178038217930768F480917B04B9
S1231A4090917C04826090937C0480937B0480917D04806836C080917B0490917C048D7F1D
S1231A600BC090919F04809179038917F0F080917B0490917C048B7F90937C0480937B0456
S1231A802BC0209191043091920421153105E1F08091590490915A048D5D9540A8F02150C8
S1231AA03040309392042093910480917B0490917C04846090937C0480937B0480917D0435
S1231AC0826080937D0408C01092940410929304109292041092910480917D0481FF07C009
S1231AE08091300180FF03C084E68093CA0480917F04853009F06DC090919F048091790353
S1231B00891708F05DC080918904823001F180918904813041F48091D30790E083709070F8
S1231B20892B69F056C0809189048823A1F48091D30790E083709070892B09F44AC0809186
S1231B401606909117068739910508F442C08AEF80935504089580918904833069F4809192
S1231B607B0490917C04846090937C0480937B0480917D04846021C080918904843069F422
S1231B8080917B0490917C04846090937C0480937B0480917D04886010C08091890485305A
S1231BA0C1F480917B0490917C04846090937C0480937B0480917D04826080937D0408957D
S1231BC080917B0490917C048B7F90937C0480937B0408959C018091F20384FF19C0C9012B
S1231BE0C2979C01B3E0220F331FBA95E1F7880F991F280F391F2455354F442737FD40955F
S1231C00542F60E579E784E090E00E94753020C08091F20385FD02C024E61AC0C901C2974C
S1231C209C01F3E0220F331FFA95E1F7880F991F280F391F2455354F442737FD4095542F74
S1231C4060E579E784E090E00E9475302C592695822F0895A89582E50E94182F83E10E949F
S1231C60182F8091590490915A04892F0E94182F8091590490915A040E94182F80910A0496
S1231C8090910B040E94182F8091D4078E5C0E94182F8091F4039091F5030E94182F80914D
S1231CA00204909103040E94182F80910004909101040E94182F8091FC039091FD030E9412
S1231CC0182F80916004909161046091180170E00E942C30862F0E94182F80915D04909135
S1231CE05E0420915F0434E0969587953A95E1F7807F822B0E94182F80915D0490915E04DE
S1231D000E94182F2091A3073091A40780911406909115068870832B0E94182F8091A3075E
S1231D209091A4070E94182F8091D1040E94182F8091C8070E94182F8091FA039091FB0325
S1231D400E94182F8091160690911706969587950E94182F86B1869586958695817090E012
S1231D609093500680934F068091B50490E0909352068093510686B18695817090E0909389
S1231D8054068093530680919D0490919E0490935606809355068091990490919A04909387
S1231DA058068093570680917B0490917C0490935A06809359068091D5039091D603909325
S1231DC05C0680935B06809140069091410690935E0680935D0680919004E82FF0E0EE0FE4
S1231DE0FF1FE15BF94F208131818295807F832B0E94182FE0919004F0E0EE0FFF1FE15B11
S1231E00F94F808191810E94182F8DEA0E94182F809190048F5F80939004883010F0109286
S1231E20900408958F929F92AF92BF92CF92DF92EF92FF920F931F93CF93DF93A89588E1D7
S1231E400FB6F89480936000109260000FBE0E94612F882311F40C94EF160E94F52E90937C
S1231E608F0480938E048236910509F47CC48336910508F04FC08D34910509F44DC38E341F
S1231E80910528F58433910511F40C94B0168533910578F48832910509F484C68932910531
S1231EA009F4AAC68132910511F00C94EF160C94C7168534910509F487C18634910509F464
S1231EC02EC28134910511F00C94EF16C1C08535910509F4EAC58635910570F4823591059E
S1231EE009F496C58335910509F4E4C68035910511F00C94EF16E6C48835910509F422C6BE
S1231F008136910509F452C08735910511F00C94EF163BC58F36910509F42BC680379105D3
S1231F20E8F48636910509F4B6C18736910548F48436910509F41DC48536910508F06DC3C5
S1231F4015C48936910509F471C48D36910509F4A2C28736910509F042C78EC48A37910565
S1231F6009F461C48B37910568F48837910509F45AC48937910508F069C68037910509F054
S1231F802EC7C7C4863F910509F426C2873F910528F4853F910509F022C79FC1873F91050D
S1231FA069F1883F910509F01AC7AFC081E60E94182F80EA0E94182F10928F0410928E0411
S1231FC00EC0EE59F94F80810E94182F80918E0490918F04019690938F0480938E04E091FC
S1231FE08E04F0918F04E03AF10558F38FEF99E50197F1F7000000C08EE927C087EF0E942A
S1232000182F80EA0E94182F10928F0410928E040EC0EE5FF84F80810E94182F80918E04CA
S123202090918F04019690938F0480938E04E0918E04F0918F04E03AF10558F38FEF99E588
S12320400197F1F7000000C088E00E94182FC7C610928F0410928E0400E010E0AFEFEA2E6F
S1232060A3EBFA2E0E94612F882309F446C0C0918E04D0918F04C03AD10579F50E94F52EEC
S123208090938F0480938E048E3B910579F481E40E94182F81E00E94182F81E00E94182F33
S12320A08EEB0E94182F06E11AEF27C081E40E94182F81E00E94182F80E00E94182F8EEB89
S12320C00E94182FC7010197F1F7000000C0E0918C04F0918D04099510C00E94F52ECE599E
S12320E0D94F888380918E0490918F04019690938F0480938E0400E010E00F5F1F4F2AEF9B
S12321000030120708F4AECF6AC610928F0410928E04C0E0D0E0FFEFEF2EF3EBFF2E0E9458
S1232120612F882309F449C000918E0410918F04003A110579F50E94F52E90938F048093B7
S12321408E048730910579F488EF0E94182F81E00E94182F81E00E94182F87E00E94182FEB
S1232160C6E1DAEF2AC088EF0E94182F81E00E94182F80E00E94182F87E00E94182FC701F6
S12321800197F1F7000000C0E0918C04F0918D04099513C000561F4F0E94F52E0E59194F1F
S12321A0F801808380918E0490918F04019690938F0480938E04C0E0D0E02196FAEFC030F6
S12321C0DF0708F4ACCF0BC6C0E0D0E0E8E1FE2E0AEF10E00E94612F882309F455C00E940E
S12321E0F52E8A3B910509F0FAC50FB6F894F0926000109260000FBE10928F0410928E043A
S12322003BC0885B0E94182F8DEF0E94182F80918E0490918F04809FE001819FD00D909F0B
S1232220D00D112409C0F999FECFD2BDC1BDF89A80B50E94182F219620918E0430918F0455
S12322402F5F3F4F209FC001219F900D309F900D112421503040C817D90728F3822F885B91
S123226080950E94182F80918E0490918F04019690938F0480938E0480918E0490918F04BC
S12322808430910508F4BDCF21962AEFC030D20708F4A0CFA4C586E60E94182F80EA0E949A
S12322A0182F10928F0410928E040EC0ED52FB4F80810E94182F80918E0490918F0401963B
S12322C090938F0480938E04E0918E04F0918F04E03AF10558F389E9B8CE85EF0E94182FD8
S12322E080EA0E94182F10928F0410928E040EC0ED58FA4F80810E94182F80918E04909114
S12323008F04019690938F0480938E04E0918E04F0918F04E03AF10558F38AE096CE109252
S12323208F0410928E0400E010E07FEFE72E73EBF72E0E94612F882309F446C0C0918E0439
S1232340D0918F04C03AD10579F50E94F52E90938F0480938E04893B910579F486E40E9454
S1232360182F81E00E94182F81E00E94182F89EB0E94182F06E11AEF27C086E40E94182FF7
S123238081E00E94182F80E00E94182F89EB0E94182FC7010197F1F7000000C0E0918C0440
S12323A0F0918D04099510C00E94F52ECD52DB4F888380918E0490918F04019690938F04DC
S12323C080938E0400E010E00F5F1F4F3AEF0030130708F4AECF03C510928F0410928E048B
S12323E0C0E0D0E06FEFE62E63EBF62E0E94612F882309F449C000918E0410918F04003A31
S1232400110579F50E94F52E90938F0480938E048930910579F486EF0E94182F81E00E94F7
S1232420182F81E00E94182F89E00E94182FC6E1DAEF2AC086EF0E94182F81E00E94182FB3
S123244080E00E94182F89E00E94182FC7010197F1F7000000C0E0918C04F0918D04099524
S123246013C000561F4F0E94F52E0D521B4FF801808380918E0490918F04019690938F0493
S123248080938E04C0E0D0E02196FAEFC030DF0708F4ACCFA4C48DE60E94182F89E00E9487
S12324A0182F80911F01909120010E94182F80911F0190912001892F0E94182F809125012A
S12324C0909126010E94182F8091250190912601892F0E94182F80910001909101010E94D0
S12324E0182F8091000190910101892F0E94182F809113010E94182F809112010E94182FA0
S1232500F999FECF89E591E092BD81BDF89A80B50E94182F82E999CD10928F0410928E0402
S1232520AA24BB245AE0852E912C0E94612F8A3008F469C00E94F52E9093200180931F01F3
S123254000911F01109120010E94F52ED82ECC240C0D1D1D1093200100931F010E94F52EBA
S1232560909326018093250100912501109126010E94F52EF82EEE240E0D1F1D1093260137
S1232580009325010E94F52E909301018093000100910001109101010E94F52ED82FC0E0DF
S12325A00C0F1D1F10930101009300010E94F52E809313010E94F52E809312010E94F52EEB
S12325C0F999FECF1FBA92BC81BC80BD0FB6F894FA9AF99A0FBE0E9461290E94F52E823B04
S12325E0910561F40E941205E0918C04F0918D0409954FE6A42E4AEFB42E05C0E0918C049A
S1232600F0918D0409950894A11CB11C20E0A2162AEFB20608F489CFE2C385E60E94182F0A
S123262083E10E94182F10928F0410928E040EC0EB51FE4F80810E94182F80918E049091DB
S12326408F04019690938F0480938E04E0918E04F0918F04EA30F10558F380911901909133
S12326601A016091180170E00E942C30862F0E94182F80911C0190911D016091180170E07E
S12326800E942C30862F0E94182F8FEF95E30197F1F7000000C080912A010E94182F80912E
S12326A02B010E94182F80912C010E94182F80912D010E94182F809114019091150166E00F
S12326C070E00E942C30862F0E94182F809127010E94182FF999FECF8EE691E092BD81BD17
S12326E0F89A80B50E94182F8AE90E94182F8CE60E94182F84E10E94182F10928F0410924A
S12327008E040EC0E75EF94F80810E94182F80918E0490918F04019690938F0480938E0495
S1232720E0918E04F0918F04EA30F10558F310928F0410928E040EC0E75EF94F80890E94B4
S1232740182F80918E0490918F04019690938F0480938E04E0918E04F0918F04EA30F105BE
S123276058F383E972CC0E94A40039C30E94D90036C381E50E94182F80E10E94182F809100
S12327809B0490919C04892F0E94182F80919B0490919C040E94182F80915F0690916006DD
S12327A0892F0E94182F80915F06909160060E94182F8091DE079091DF070E94182F809197
S12327C0E0079091E1070E94182F8091990490919A040E94182F8091FC039091FD030E94F3
S12327E0182F80917D040E94182F80917B0490917C040E94182F8091EE0780950E94182FF5
S123280080919F040E94182F809139060E94182F84E00E94182F85E00E94182F86E00E943B
S1232820182F8EEA12CC0E942A0ED9C20E94612F8530E0F30E94F52EC82FD0E00E94F52E97
S1232840C817D90709F0CBC20E94F52E8C0190938F0480938E040E94F52E0817190709F085
S1232860BEC20E94F52E8639910509F0B8C280918E04CE59D94F4BC00E94612F8530E0F390
S12328800E94F52EC82FD0E00E94F52EC817D90709F0A5C20E94F52E8C0190938F048093C9
S12328A08E040E94F52E0817190709F098C20E94F52E8839910509F092C280918E04CD5200
S12328C0DB4F25C00E94612F8530E0F30E94F52EC82FD0E00E94F52EC817D90709F07FC201
S12328E00E94F52E8C0190938F0480938E040E94F52E0817190709F072C20E94F52E8F3A68
S1232900910509F06CC280918E04CB5BDE4F888366C2C0E0D0E00E94612F823080F10E9486
S1232920F52E0E94F52E8F38910509F058C210928F0410928E041CC0EB5BFE4F108180E76B
S12329400E94182F82E00E94182F80918E040E94182F812F0E94182F8FE80E94182F8091A9
S12329608E0490918F04019690938F0480938E04E0918E04F0918F04E03AF105E8F2219663
S12329803AEFC030D30739F62AC20E94612F8530E0F30E94F52EE82ED92E0E94F52EF82E9E
S12329A00E94F52E8C0190938F0480938E040E94F52E0817190709F012C28E2D9D2DDF2D04
S12329C0C0E08E01080F191F0E94F52E883A9105C9F4C80161E670E00E94D62FBC01607007
S12329E080918E0490918F04682B792B70938F0460938E04C80149E650E00E94EC2F12BC77
S1232A0011BCEDC1E0918C04F0918D040995BDCFAA24BB240E94612F833008F43CC00E94CE
S1232A20F52E082F992E0E94F52E182F0E94F52E8D3A910509F0D3C1F999FECF802F992DE2
S1232A40D12ECC24E601C80FD91FD2BDC1BDF89A90B5F999FECF2196D2BDC1BD2197F89A7C
S1232A6080B5F82EEE248701090F111D84E50E94182F84E00E94182F802F0E94182F8C2F25
S1232A800E94182F8D2F0E94182F812F0E94182F8BEA0E94182F0894A11CB11C80E0A81669
S1232AA08AEFB80609F0B6CF9AC1AA24BB240E94612F833008F43CC00E94F52E082F992EB5
S1232AC00E94F52E182F0E94F52E8A3A910509F086C1F999FECF802F992DD12ECC24E601DD
S1232AE0C80FD91FD2BDC1BDF89A90B5F999FECF2196D2BDC1BD2197F89A80B5F82EEE2445
S1232B008701090F111D85E50E94182F84E00E94182F802F0E94182F812F0E94182F8C2F57
S1232B200E94182F8D2F0E94182F8AEA0E94182F0894A11CB11CE0E0AE16EAEFBE0609F066
S1232B40B6CF4DC1C0E0D0E00E94612F882359F00E94F52E873A910509F041C1E0918C0450
S1232B60F0918D0409952196FAEFC030DF0761F736C1C0E0D0E00E94612F882369F00E94B4
S1232B80F52E8039910509F02AC10E940B01E0918C04F0918D04099521962AEFC030D207E3
S1232BA051F71DC1C0E0D0E00DE611E00E94612F8823E1F00E94F52E873D910509F00FC121
S1232BC08091000490910104F999FECF1FBA12BD01BD80BD0FB6F894FA9AF99A0FBE12BCA1
S1232BE011BCE0918C04F0918D04099521963AEFC030D307D9F6F3C0C0E0D0E00EE611E0F2
S1232C000E94612F8823E1F00E94F52E863D910509F0E5C08091000490910104F999FECFAC
S1232C201FBA12BD01BD80BD0FB6F894FA9AF99A0FBE12BC11BCE0918C04F0918D0409955C
S1232C4021968AEFC030D807D9F6C9C0C0E0D0E00E94612F823040F10E94F52E892B09F042
S1232C60BEC00E94F52E86389105F1F489E70E94182F87E00E94182F8FEC0E94182F8FE355
S1232C800E94182F88E00E94182F87EA0E94182F85ED0E94182F84E10E94182F80E10E94F0
S1232CA0182F86E80E94182F2196EAEFC030DE0779F695C0C0E0D0E00E94612F823008F419
S1232CC048C00E94F52E892B09F043C00E94F52E8C3A910509F083C083E50E94182F88E05D
S1232CE00E94182F80919B0490919C040E94182F80919B0490919C04892F0E94182F80916A
S1232D005F06909160060E94182F80915F0690916006892F0E94182F8091C0049091C10481
S1232D200E94182F8091C0049091C104892F0E94182F8091F4079091F5070E94182F809127
S1232D40F4079091F507892F0E94182F8CEA0E94182F2196FAEFC030DF0709F0ADCF3FC06D
S1232D60C0E0D0E00E94612F823058F00E94F52E892BA9F50E94F52E8B3C910511F40E94F3
S1232D80260121962AEFC030D20761F728C0C0E0D0E004E610E00E94612F8330D8F00E94B6
S1232DA0F52E0197E1F40E94F52EFC01E09FC001E19F900DF09F900D112490938B0480933A
S1232DC08A040E94F52E8E3D910521F010928B0410928A042196FAEFC030DF07E1F6A8953F
S1232DE0DF91CF911F910F91FF90EF90DF90CF90BF90AF909F908F900895CF93DF93CFEFC8
S1232E00D3E222C0CE010197F1F7000000C00E94120F2D982C9ACE010197F1F7000000C0AB
S1232E2081E20E94182F80E00E94182F8EED0E94182F2D9A2C9880918A0490918B04019723
S1232E4090938B0480938A0480918A0490918B040B97C0F62D9A2C9A10928B0410928A0486
S1232E60DF91CF9108952F923F924F925F926F927F928F929F92AF92BF92CF92DF92EF9234
S1232E80FF920F931F93CF93DF9314BEA89588E10FB6F89480936000109260000FBE1092C8
S1232EA0A4071092A3070E94632E259A249A209A219A2D9A2C9A289A299A579A5F9A0000F6
S1232EC000000000000081E08093D0048093CC078093D20480936106549A559A5C9A5D9A93
S1232EE0229A239A569A2A9A2B985E980000000052983A983B98439A3A98429A3998419A22
S1232F003898409A0E946A2EF999FECF8AE591E092BD81BDF89A80B5809368040E94481EAF
S1232F200E9461290E94532E10927A0010927C0080E880BF87EE80937A0011B885E090E0BD
S1232F40909301048093000488E790E09093F5038093F40384E690E090930304809302040D
S1232F6090930B0480930A0486E490E090930504809304040E942D072A9A2B98F999FECF1D
S1232F8087E090E092BD81BDF89A80B512BC11BC85FFEEC080910001909101019F7D9093C1
S1232FA00101809300010E9412050E9499050E94D9000E94A4000E940B01F999FECF1FBA57
S1232FC08AE090E092BD81BD86E080BD0FB6F894FA9AF99A0FBEF999FECF1FBA8BE090E08B
S1232FE092BD81BD89E180BD0FB6F894FA9AF99A0FBEF999FECF1FBA8CE090E092BD81BDB3
S12330008EE180BD0FB6F894FA9AF99A0FBEF999FECF1FBA8EE090E092BD81BD8EE180BD6C
S12330200FB6F894FA9AF99A0FBE80E090E0FC01EB51FE4FE081F999FECF1FBA825A9E4F8F
S123304092BD81BDE0BD0FB6F894FA9AF99A0FBE8D5591408A30910551F780E090E0FC01E5
S1233060E65DFE4FE081F999FECF1FBA87599E4F92BD81BDE0BD0FB6F894FA9AF99A0FBEE7
S1233080885691408430910551F780E090E0FC01E75EF94FE081F999FECF1FBA8E589E4F25
S12330A092BD81BDE0BD0FB6F894FA9AF99A0FBE815791408A30910551F780E090E0FC018F
S12330C0E75EF94F2089F999FECF1FBA84589E4F92BD81BD20BD0FB6F894FA9AF99A0FBE06
S12330E08B5791408A30910551F720913C06F999FECF1FBA81E791E092BD81BD20BD0FB64E
S1233100F894FA9AF99A0FBE2091140130911501F999FECF1FBA8DE090E092BD81BDC90122
S123312066E070E00E942C3060BD0FB6F894FA9AF99A0FBEF999FECF1FBA8DE691E092BD2A
S123314081BD84E180BD0FB6F894FA9AF99A0FBEF999FECF1FBA8EE691E092BD81BD81EE2D
S123316080BD0FB6F894FA9AF99A0FBE12BC11BC0E94F3000E94260120E030E0F999FECF61
S1233180205F3F4F32BD21BD20513040F89A80B5F901ED52FB4F80832F5F3F4F81E0203452
S12331A0380761F712BC11BC0E947600809100019091010185FD07C080916F008B7F8093A6
S12331C06F002D9A2C9A80912901882311F480E801C080E480933B011092F303809114016A
S12331E0909115018D5A9D4030F08CEA9DE090931501809314011092560486B3866086BB00
S123320078948AEA0E94182F80E00E94182F85E50E94182F86B18695817080936A048091D0
S12332206E00836080936E002A9AFF24F394F4E0BF2EE6E0AE2E72E4972E65E0862E57E894
S1233240752E47E0642E33E4532E26E4422E9BE4C92ED12C83E0382E04E4202E14E6E12E81
S1233260A8958091590490915A048635910598F180915604882379F58091990490919A0455
S1233280029748F18091A3079091A4079F7E9093A4078093A30780916F00856080936F0042
S12332A080916E00836080936E002A9AF09256048091A3079091A40780629093A40780933D
S12332C0A3078091A3079091A40790629093A4078093A30758C080915604813009F053C0FC
S12332E08091590490915A048234910538F08091990490919A04892B09F045C080916F00CA
S12333008D7F80936F00809170008C7F8093700080916F008B7F80936F0080916E0083609E
S123332080936E008091A3079091A4078F7D9093A4078093A3078091A3079091A407877F5D
S12333409093A4078093A307F092D004F092CC07F092D204F09261065C9A5D9A2D9A2C9A78
S1233360289A299A109256048091A3079091A4079F7D9093A4078093A307109254041092FE
S12333809A041092990480915604813001F580916F00826080936F008091700083608093DF
S12333A07000B5BC80916E00836080936E008091A3079091A40788609093A4078093A3074B
S12333C02A9A2B9A10928B0410928A0420C015BC109254042D9A2C9A289A299A2B981092DD
S12333E054041092B30010926104109260048091430190914401892B51F42A9880918A04FA
S123340090918B048536910510F00E94FD168091F303833009F4CFC0843018F4882371F0E0
S123342074C0853009F4ECC1853008F427C1863009F49DC1873009F06AC223C2809157041E
S1233440909158048536910508F463C2E091F303F0E080917800909179008C7F65E070E07F
S12334600E942C30EE0FFF1FEC5CFB4F718360838091F303C82FD0E0E091F303F0E0EE0FE4
S1233480FF1FEC50FC4F80819181E091F303F0E0EE0FFF1FEC5CFB4F20813181880F991FEA
S12334A0880F991F820F931F880F991F6AE070E00E942C30CC0FDD1FCC50DC4F798368838A
S12334C01092580410925704F092F30381E480937C000E94120F809114019091150190933E
S12334E01701809316018091430190914401892B51F080914301909144010197909344011B
S1233500809343012A9AA89504C280915704909158048536910508F4FCC1109258041092F6
S12335205704A8958091F303813041F580910801909109012091780030917900820F931F16
S123354096958795909309018093080183E00E9429099093F7038093F6038091F60390914C
S1233560F70390930B0480930A04E092CD0722E02093F30385E480937C00CBC18091020171
S1233580909103012091780030917900820F931F969587959093030180930201D092F9037A
S12335A0C092F803D0920504C09204043092F30320927C00AEC180915704909158048536FC
S12335C0910508F4A6C1E091F303F0E080917800909179009695879596958795EE0FFF1FEB
S12335E0EC5CFB4F918380838091F303C82FD0E0E091F303F0E0EE0FFF1FEC50FC4F808196
S12336009181E091F303F0E0EE0FFF1FEC5CFB4F20813181880F991F880F991F820F931F7C
S1233620880F991F6AE070E00E942C30CB01CC0FDD1FCC50DC4F99838883109258041092EE
S12336405704B092F30380913B0180937C000E94120FA89580917A048F5F80937A04843035
S123366010F010927A0480917A04982F91709093C4048695817080933F064BC18091570408
S1233680909158048159914008F443C180912901882329F1E091F303F0E08091780090911D
S12336A079009695879596958795EE0FFF1FEC5CFB4F91838083A091F303B0E0E091F3031D
S12336C0F0E0EE0FFF1FEC5CFB4F80819181AA0FBB1FAC50BC4F11969C938E933EC0E09156
S12336E0F303F0E08091780090917900EE0FFF1FEC5CFB4F918380838091F303C82FD0E06B
S1233700E091F303F0E0EE0FFF1FEC50FC4F00811181E091F303F0E0EE0FFF1FEC5CFB4FD5
S1233720808191810E941A0A9C01220F331F280F391FC801F3E0880F991FFA95E1F7801B10
S1233740910B820F931F6AE070E00E942C30CC0FDD1FCC50DC4F7983688310925804109249
S123376057048092F30370927C00A895D2C080915704909158048536910508F4CAC0E09164
S1233780F303F0E080917800909179009695879596958795EE0FFF1FEC5CFB4F91838083EA
S12337A0A091F303B0E0E091F303F0E0EE0FFF1FEC50FC4F20813181E091F303F0E0EE0FEE
S12337C0FF1FEC5CFB4F80819181820F931F880F991F9695879596958795AA0FBB1FAC5073
S12337E0BC4F11969C938E9310925804109257046092F30350927C000E94120FA89589C039
S12338008091570490915804893C910508F481C0E091F303F0E08091780090917900EE0FCC
S1233820FF1FEC5CFB4F91838083A091F303B0E0E091F303F0E0EE0FFF1FEC50FC4F20818C
S12338403181E091F303F0E0EE0FFF1FEC5CFB4F80819181820F931F96958795AA0FBB1F9E
S1233860AC50BC4F11969C938E931092580410925704A092F30390927C000E94120FA89585
S123388048C080915704909158048536910508F440C0E091F303F0E080917800909179008C
S12338A0969587959695879590E0EE0FFF1FEC5CFB4F91838083A091F303B0E0E091F30324
S12338C0F0E0EE0FFF1FEC50FC4F20813181E091F303F0E0EE0FFF1FEC5CFB4F8081918128
S12338E0820F931F96958795AA0FBB1FAC50BC4F11969C938E93109258041092570410920C
S1233900F30340927C000E94120FA89502C0F092F303809157049091580401969093580426
S1233920809357048091590490915A048F55914008F448C08091FA0787FF02C0E0E002C093
S1233940E091FA078091CA078F5F8093CA079091CA078091CB079817B8F11092CA072091EC
S1233960020430910304AE2FB0E0FD01E855F84F808190E02817390754F48091C8078436B4
S123398034F48091C8079091C907890F12C02091020430910304A855B84F8C9190E0281771
S12339A039074CF08091C80782302CF08091C80781508093C8078091C80785362CF0E0921D
S12339C0C80702C0F092C8078091590490915A048739910508F46DC08091270120910004A7
S12339E03091010490E04896821793070CF461C08091CC049091CD0401969093CD048093EA
S1233A00CC042091CC043091CD048091CE049091CF042817390708F440C01092CD04109258
S1233A20CC042091590430915A048091C6049091C7040A972817390730F49091CA0480917A
S1233A40CB04890F15C02091590430915A048091C6049091C70449968217930758F49091B3
S1233A60CA048091C904891728F48091CA0481508093CA049091CA048091C804891718F4D1
S1233A808091C80408C09091CA048091C904981720F48091C9048093CA048091590490919F
S1233AA05A048A58924038F48091C8048093CA0402C01092CA048091F20382FF55C0809127
S1233AC0590490915A04855F914008F44DC08091590490915A04805D974008F045C0809199
S1233AE02701209100043091010490E0049682179307D4F1209100043091010480916D0420
S1233B0090E00196821793077CF180910A0490910B048F36910544F180916E0490916F0404
S1233B20A0917004B09171040196A11DB11D80936E0490936F04A0937004B0937104809178
S1233B406E0490916F04A0917004B091710481549D40A340B04008F1F0926C048091A307D5
S1233B609091A407916015C0809100049091010480936D0410926E0410926F0410927004B1
S1233B801092710410926C048091A3079091A4079E7F9093A4078093A3070E944D0B0E942D
S1233BA0750C0E94860A809100019091010180FF67C08091300180FF11C08091BE04883C4A
S1233BC028F08091CA048823C9F016C09091CA048091BE048695891790F010C080913001A1
S1233BE082FF0DC08091BE04883C48F08091A3079091A40796FF02C05C9A01C05C9880910A
S1233C00300184FF16C08091BE04883C28F08091C80718165CF12CC02091C8078091BE04CD
S1233C20332727FD3095869590E0821793070CF11FC08091300186FF1CC08091BE04883C69
S1233C40C0F02091590430915A0480913501909136018217930760F42091020430910304DE
S1233C608091690490E08217930714F45D9A01C05D988091BE04883C28F01092BE0402C095
S1233C805C9A5D9A8091BE048F5F8093BE04E8CA1092800081EF9FEF909389008093880084
S1233CA085EF9FEF90938B0080938A0080E88093810080EC9AED909385008093840083E022
S1233CC090E09093D6038093D5038091D5039091D60380688093810010925A04109259042B
S1233CE080916F00876080936F0052983A98259A249A2D9A2C9A289A299AF999FECF82E0CB
S1233D0092E092BD81BDF89A80B58093BA03F999FECF81E092E092BD81BDF89A80B5809370
S1233D20BB038091BB038E3039F08091BB03873119F087E18093BB038091690081608093D4
S1233D406900E89A84E08093680080936D0008951F920F920FB60F9211242F933F938F93D5
S1233D609F9386B18695869581702091680490E030E08217930789F581E08093B504809123
S1233D80D4078230E9F48091640490916504880F991F9093650480936404809164049091C2
S1233DA06504816090936504809364048091990490919A04019690939A04809399040DC06C
S1233DC08091990490919A04019790939A048093990410926504109264049F918F913F9134
S1233DE02F910F900FBE0F901F9018951F920F920FB60F9211248F939F938091FB078F5F56
S1233E008093FB078091FB07882309F44DC08091A3079091A40790619093A4078093A307BE
S1233E20109256048091A3079091A4079F7D9093A4078093A30780916F008B7F80936F0048
S1233E4080916F008D7F80936F00809170008C7F8093700080916E00836080936E002D9A97
S1233E602C9A289A299A8091A3079091A4078F7D9093A4078093A3078091A3079091A4074E
S1233E80877F9093A4078093A30781E08093D0048093CC078093D204809361065C9A5D9A0F
S1233EA010925A041092590410929A041092990478949F918F910F900FBE0F901F901895BD
S1233EC08091B504813091F41092B50483E08093D4078091B6039091B7039093B90380939B
S1233EE0B8031092B7031092B6031FC08091D4078F5F8093D4078091D407853019F481E096
S1233F008093D4078091D407833079F48091990490919A04892B49F08091990490919A04DC
S1233F20019790939A04809399048091990490919A04069730F085E090E090939A048093A1
S1233F40990480918400909185009093F9078093F80708951F920F920FB60F9211248F93A4
S1233F609F938091B6039091B70301969093B7038093B6039F918F910F900FBE0F901F901C
S1233F8018958091A3079091A40793FD17C08091D407813011F42D9808958091D4078430DE
S1233FA011F42C9808958091D407823011F4289808958091D407833009F4299808951F93EB
S1233FC08091B604882309F4B1C08091B604813091F48091590490915A048955924010F05B
S1233FE02D9A299A8091B6039091B703909307088093060815C08091B604823089F480915B
S1234000590490915A048955924010F02C9A289A8091B6039091B7039093ED078093EC07C6
S12340208091B704882359F48091590490915A048955924008F467C01092B60464C0809167
S1234040B704813099F480918A0090918B004E9690938B0080938A008091B6048C5980932A
S1234060B6048091B6048093B7044DC08091B704853611F585B190E2892785B980918A001E
S123408090918B004E9690938B0080938A00209102083091030840910408509105088091DE
S12340A08A0090918B00A0E0B0E0281739074A075B0748F52D9A25C08091B704863619F505
S12340C085B190E1892785B980918A0090918B004E9690938B0080938A0020910208309155
S12340E00308409104085091050880918A0090918B00A0E0B0E0281739074A075B0718F451
S12341002C9A1092B70480913D0690913E06892B49F18091F607882329F180913D06909189
S12341203E0690938B0080938A001CC08091F6078823C1F01091F607113021F01091F60718
S1234140123031F48091F6070E94C11F1093B6048091F4079091F50790938B0080938A0093
S12341601092F6071F9108951F920F920FB60F9211242F933F934F935F936F937F938F93C4
S12341809F93AF93BF93EF93FF930E94DF1F2A9A7894FF91EF91BF91AF919F918F917F91D1
S12341A06F915F914F913F912F910F900FBE0F901F9018951F920F920FB60F9211248F9325
S12341C09F93F8948091D507882309F492C080917B0490917C0497FD8CC0809113018095EB
S12341E08093EE078091EE07909139068C59891B8093EE0790911806943071F1953040F45E
S12342009230C1F19330D8F4913009F072C00AC0973109F44CC0933609F457C09E3009F06C
S123422068C035C08091EE078093B20084E08093B1001092D0049093C30483E018C08091BE
S1234240EE078093B20094E09093B1001092D20483E08093C3044BC08091EE078093B200CD
S12342609093B100109261069093C30482E0809318063FC08091EE078093B20084E080939F
S1234280B1001092CC079093C30481E0F0CF81E08093DA038091EE078093B20084E0809357
S12342A0B1001092D0041092610687E1E0CF81E08093DB038091EE0786BD83E085BD1092D1
S12342C0CC071092D2048EE0D2CF81E08093DA038091EE078093B20084E08093B10010929A
S12342E0D004109261061092D2041092CC079093180678949F918F910F900FBE0F901F9099
S12343001895EF92FF920F931F93CF93DF93EC0180916704E7E0F0E0E81BF109EE0FFF1F9A
S1234320EC50FC4F0190F081E02D80916604E81BF109F7FF02C0E0E0F0E080912E0126E0DD
S1234340829FC00111249C012E9FC0012F9F900D3E9F900D112464E670E00E944030CB0185
S1234360603A71050CF08FE98093F7078091F7076AE00E9420308093D0078091D0078031D6
S12343801CF08FE08093D0078091590490915A04885E934008F0AAC01092CE078FEF8093A4
S12343A0FA078091D00724E18202C001112490935E0480935D048091590490915A0464E661
S12343C070E00E942C3065506093F3078091590490915A04845F914060F41092F307E091E7
S12343E0F307FF27E7FDF095E25CFE4F808190E0A9C08091F3078430E1F5E0915D04F091E3
S12344005E04EE59F94F2081E091F307FF27E7FDF095E25CFE4F6081E091F307FF27E7FD2B
S1234420F095E25CFE4F808190E09093170680931606E0911606F0911706809159049091CE
S12344405A044091F30730E0220F331F261B3109845F91406CE94602A0011124840F951FB3
S1234460AC01249FC001259F900D349F900D11243AC0E091F307FF27E7FDF095E15CFE4F83
S12344806081E091F307FF27E7FDF095E25CFE4F4081E091F307FF27E7FDF095E25CFE4F6C
S12344A0808190E09093170680931606E0911606F09117068091590490915A042091F30755
S12344C070E0641B7109845F91404CE9240290011124820F931F9C01629FC001639F900D79
S12344E0729F900D112464E670E0D1C08091590490915A04815A984250F187EC8093CE076C
S12345008091CE076AE00E9420308093FA078091D0072091FA0744E18402C00111243327CC
S123452027FD3095820F931F90935E0480935D04E0915D04F0915E04EE59F94F808190E09D
S1234540880F991F9093170680931606A8C08091590490915A04885E934062E370E00E9454
S12345602C306093CE078091CE076AE00E9420308093FA078091D0072091FA0744E1840298
S1234580C0011124332727FD3095820F931F90935E0480935D04E0915D04F0915E04EE59A6
S12345A0F94F808190E0880F991F90931706809316068091FA0787FD37C08091FA0783312D
S12345C09CF5E0915D04F0915E04ED59F94F4081E0915D04F0915E04EE59F94F6081E091AC
S12345E01606F09117063091CE078091FA0726EF8202C0011124830F911D880F991F50E007
S1234600461B51099C01249FC001259F900D349F900D11246AE070E00E944030E60FF71FFD
S1234620F0931706E09316068091D00787FD37C08091D0078F309CF5E0915D04F0915E04F7
S1234640EA58F94F4081E0915D04F0915E04EE59F94F6081E0911606F09117063091F707FC
S12346608091D00726EF8202C0011124830F911D880F991F50E0461B51099C01249FC00124
S1234680259F900D349F900D11246AE070E00E944030E60FF71FF0931706E0931606809119
S12346A0A3079091A407977F9093A4078093A3078091140690911506877F90931506809321
S12346C0140680917D04882309F458C080917D0487FD27C080917D04883088F08091D307C0
S12346E090E083709070892B09F448C08091D30767E00E942030992309F440C012C08091DA
S12347007D048430C0F08091D30790E083709070892B39F08091D30767E00E9420309923A5
S123472069F58091A3079091A40798609093A4078093A30723C080917D04823050F0809195
S12347401406909115068860909315068093140615C080917D04882389F0809116069091D3
S123476017068739910550F080911606909117068C58904090931706809316068091D30709
S12347808F5F8093D30790919F04945695310CF094E1209116063091170680915504281BFD
S12347A03109892F9C3E0CF48CEE992787FD9095280F391F30939E0420939D0480919D044C
S12347C090919E04909317068093160680911606909117062091120180589040820F911D8D
S12347E090939E0480939D0420919D0430919E048091BF044AE08402C0011124820F931FCA
S123480090939E0480939D04809112012091BF0490E080589F4F240290011124820F931F1E
S1234820AC014C9FC0014D9F900D5C9F900D1124A0E0B0E08093020890930308A09304082B
S1234840B09305086091020870910308809104089091050828E037E040E050E00E9453301E
S1234860C901DA018093020890930308A0930408B093050880919D0490919E048D5B924086
S12348803CF04CEBE42E42E0F42E012D112D15C080919D0490919E04059734F435E0E32EBB
S12348A0F12C012D112D09C080919D0490919E047C010027F7FC0095102FF0929E04E0922C
S12348C09D0420915B0430915C042C0F3D1F40E050E0C801B7010E94013028E037E040E088
S12348E050E00E945330CE01821B930BDF91CF911F910F91FF90EF9008950F931F93209185
S12349009D0430919E04442737FD4095542FBC0176956795680F791F70939C0460939B0490
S123492060919B0470919C0480E090E00E94013000919B0410919C0428E037E040E050E0BF
S12349400E945330021B130BC8011F910F910895DC018091FA078F302CF02FE030E040E034
S123496050E00BC08091FA07992787FD909501969C01442737FD4095542FF901E454FC4F15
S1234980608170E080E090E09D0140E050E00E94013028E037E040E050E00E945330C901F3
S12349A008950F931F93CF93DF938091CC039091CD0390930108809300088091CC03909115
S12349C0CD03499708F46AC28091FB07882349F088EE9DEF9093D8038093D7031092FB0773
S12349E053C08091590490915A044091D7035091D803895B9B40C0F0E0915B04F0915C042C
S1234A002091CC033091CD038091BA0390E0241B350BAC01429FC001439F900D529F900D68
S1234A20112464E170E017C0E0915B04F0915C042091CC033091CD038091BA0390E0241B92
S1234A40350BAC01429FC001439F900D529F900D11246EE170E00E944030CB018E0F9F1FA9
S1234A6062E070E00E94403070935C0460935B0410925C0410925B048091CC039091CD0305
S1234A809093D8038093D70380915404893628F4809154048F5F809354048091D407813084
S1234AA029F42D9903C02D9A1092B6048091D407843029F42C9903C02C9A1092B6048091B1
S1234AC0D407823029F4289903C0289A1092B6048091D407833029F4299903C0299A1092E0
S1234AE0B6048091590490915A04C091D703D091D803D0936006C0935F0620915F0630914C
S1234B0060060091D5031091D60340E050E060E070E489E191E00E947530CA01B9012EE1AE
S1234B2030E040E050E00E94013020EC30E0A901049F9001059F300D149F300D11242050CE
S1234B40324040E050E00E94533030935A04209359042091AC043091AD044091AA04509106
S1234B60AB04C901880F991F820F931F840F951F96958795969587959093AD048093AC04BA
S1234B808091A8049091A9049093AB048093AA048091A6049091A7049093A9048093A804DD
S1234BA08091A4049091A5049093A7048093A6048091A2049091A3049093A5048093A404DD
S1234BC08091A0049091A1049093A3048093A2048091590490915A049093A1048093A00467
S1234BE08091590490915A048D5D9540B8F080919F044091A0045091A1042091AC0430918C
S1234C00AD0490E0821B930B840F951F9695879596958795855B80939F040FC084E680937D
S1234C209F0480915B0490915C0464E070E00E94403070935C0460935B041092FB078091CC
S1234C40590490915A048C529140A0F58091D5039091D603039771F58091D407813051F56A
S1234C6084E090E09093D6038093D5038091D5039091D60380688093810080918400909160
S1234C80850096958795969587959093850080938400D695C795D695C795D093D803C0939F
S1234CA0D70380915F069091600696958795969587953AC08091590490915A048F5E9240E5
S1234CC0B8F18091D5039091D603049789F58091D407813069F583E090E09093D60380934E
S1234CE0D5038091D5039091D6038068809381008091840090918500880F991F880F991FA0
S1234D009093850080938400CC0FDD1FCC0FDD1FD093D803C093D70380915F06909160063A
S1234D20880F991F880F991F9093600680935F0680915F06909160060E9481219093F50770
S1234D408093F407809114069091150683FF3AC0E091B804F091B904CF0183709070892B7C
S1234D6099F420915F063091600680915F06909160066AE070E00E942C30261B370B30938A
S1234D80F5072093F40718C020913C0180915F069091600668E270E00E942C3030E0629FF9
S1234DA0C001639F900D729F900D11248C599F4F9093F5078093F4073196F093B904E09332
S1234DC0B80404C01092B9041092B8048091590490915A048A58924038F08091F4039091A0
S1234DE0F5038E3691053CF48CE291E09093FF078093FE0704C01092FF071092FE078091E9
S1234E00F4079091F50720911601309117014091FE075091FF07821B930B841B950B90937B
S1234E20EB078093EA078091EA079091EB0797FF20C08091EA079091EB0720915F06309101
S1234E4060064091F4075091F507820F931F8417950778F48091F4079091F50720915F061A
S1234E60309160064496821B930B9093EB078093EA07F8948091D407823019F481E080932E
S1234E80180680915F06909160060E94A824909389008093880081E08093D5077894DF9172
S1234EA0CF911F910F9108951F920F920FB60F9211242F933F934F935F936F937F938F9316
S1234EC09F93AF93BF93EF93FF93F89489B18695869581702091680490E030E08217930737
S1234EE009F43DC020918400309185008091CC039091CD039695879596958795281739075B
S1234F0040F481E090E090936304809362047894C6C1789480918400909185009093CD03B8
S1234F208093CC0310928500109284000E94D1240E94601F8091620490916304880F991F38
S1234F4090936304809362048091620490916304816090936304809362045F983BC089B13B
S1234F608695869581702091680490E030E08217930781F580918400909185009093C1049D
S1234F808093C0048091590490915A048852934208F085C180918400909185000E947D24DE
S1234FA09093C1048093C0048091C0049091C1049093F5078093F4078091B604882309F4D3
S1234FC06EC18091F4079091F50790938B0080938A0065C1809114069091150683FF89C0D2
S1234FE078948091620490916304880F991F90936304809362045F9A20913C0180915F06F3
S12350009091600668E270E00E942C3030E0629FC001639F900D729F900D11248C599F4F46
S12350209093F5078093F4078091590490915A048051974208F049C08091A3079091A40720
S123504093FD43C08091F4079091F50790938B0080938A0020915F063091600680915F0692
S1235060909160069695879596958795281B390B30933E0620933D068091D407813021F0E5
S12350808091D407833031F42C9882E08093B60481E00DC08091D407843021F08091D4078A
S12350A0823039F42D9881E08093B60482E08093F6078EEB90E090934106809340068091EB
S12350C0A3079091A4079F770FC080915F06909160068C509E4F90938B0080938A0080914F
S12350E0A3079091A40790689093A4078093A307D5C078948091620490916304880F991FC4
S123510090936304809362045F9A8091590490915A048051974208F0B7C08091EA07909166
S1235120EB0785369105ECF11092B6048091590490915A048C5D954040F48091F20381FF8A
S123514004C081E08093B70402C01092B7048091EA079091EB0790938B0080938A008091C8
S12351608A0090918B0090933E0680933D068091D407813021F08091D407833011F481E085
S123518009C08091D407843021F08091D407823029F482E08093F6071092B60484E090E034
S12351A06EC08091EA079091EB078B5B9F4F8CF11092B60488EC90E090938B0080938A00CC
S12351C084E690E090933E0680933D068091D407813021F08091D407833011F481E009C0B8
S12351E08091D407843021F08091D407823039F482E08093F6070E94C11F1092B60488E275
S123520090E0909341068093400684E18093D90345C08091F4079091F50790938B00809314
S12352208A0020915F06309160068091EA079091EB07820F931F90933E0680933D0680917D
S1235240D407813021F08091D407833029F481E00E94C11F81E00CC08091D407843021F030
S12352608091D407823031F482E00E94C11F82E08093B60484E18093D90384EB90E09093FE
S12352804106809340060AC080915F06909160068C509E4F90938B0080938A002A9A7894BF
S12352A0FF91EF91BF91AF919F918F917F916F915F914F913F912F910F900FBE0F901F90D0
S12352C0189521EB30E0F90110821092B6001092B2001092B300A0E7B0E08C9183608C933E
S12352E0000000000000000081E08093D0048093CC078093D20480936106EFE6F0E0808173
S12353008D7F80838C918C7F8C93F901108215BC84E68093390608951F920F920FB60F92C5
S123532011240F900FBE0F901F901895813049F48093D00486B590E090935806809357065C
S12353400895823021F481E08093CC070895833021F481E08093D2040895843019F481E030
S12353608093610608950F931F938091590490915A04845F914018F41092F30716C080918E
S1235380590490915A048D56974020F08EE08093F3070BC08091590490915A0464E670E096
S12353A00E942C3065506093F307E091F307F0E0E151FE4F80818093130180916C0488233B
S12353C029F02091E7048091180109C0E0915D04F0915E04ED52FB4F808120911801829FF7
S12353E0C00111249093BC048093BB048091590490915A04825C914060F5809100019091DA
S1235400010182FF1CC08091BB049091BC042091190130911A01820F931F9093BC04809398
S1235420BB048091A3079091A40784609093A4078093A30780911B018093BA0444C08091A0
S1235440A3079091A4078B7F9093A4078093A3073AC08091A3079091A4078B7F9093A407E4
S12354608093A3078091BA04823068F18091BA0481508093BA042091BB043091BC0440915E
S1235480190150911A01E0911901F0911A0180911B017091BA0460911B01240F351F90E0DB
S12354A0871B9109AC014E9FC0014F9F900D5E9F900D112470E00E942C30261B370B309363
S12354C0BC042093BB0480916C04882309F0E8C08091FA0787FD3FC08091FA078331DCF59D
S12354E0E0915D04F0915E04EC52FB4F4081E0915D04F0915E04ED52FB4F20810091BB047B
S12355001091BC043091CE078091FA07E091180150E0421B510926EF8202C0011124830FEC
S1235520911D9C01429FC001439F900D529F900D11246AE070E00E944030F0E06E9FC001EE
S12355406F9F900D7E9F900D1124800F911F9093BC048093BB048091D00787FD3FC080913D
S1235560D0078F30DCF5E0915D04F0915E04E951FB4F4081E0915D04F0915E04ED52FB4F88
S123558020810091BB041091BC043091F7078091D007E091180150E0421B510926EF820204
S12355A0C0011124830F911D9C01429FC001439F900D529F900D11246AE070E00E94403084
S12355C0F0E06E9FC0016F9F900D7E9F900D1124800F911F9093BC048093BB048091000189
S12355E09091010184FF5CC02091200430912104809100049091010428173907FCF480916F
S12356000004909101042091200430912104821B930B64E070E00E94403080915F048617AF
S123562010F460935F0480915F048A3018F089E080935F04809128018093BD043091BD0467
S12356403430C8F08091BB049091BC04E0915F04F0E0EB51FE4F2081820F911D9093BC0489
S12356608093BB0431503093BD048091A3079091A407806109C010925F041092BD048091A5
S1235680A3079091A4078F7E9093A4078093A307809100049091010490932104809320043E
S12356A0809100019091010191FD09C08091F20386FF94C080916C04882309F48FC08091F2
S12356C03B068F5F80933B0690913B0680913C06981708F486C010923B068091FC03909189
S12356E0FD03E091D007FF27E7FDF095E75EF94F208130E02817390734F480913906909179
S12357003A06890F19C08091FC039091FD03E091D007FF27E7FDF095E75EF94F208130E08E
S1235720821793075CF48091390618163CF48091390690913A06891B809339068091A307D2
S12357409091A4079D7F9093A4078093A30720913906E091D007FF27E7FDF095E75EF94F7E
S12357608089332727FD309590E08C599F4F8217930754F4E091D007FF27E7FDF095E75EFF
S1235780F94F80898C591EC020913906E091D007FF27E7FDF095E75EF94F4089332727FD56
S12357A0309584E690E0841B910928173907CCF4E091D007FF27E7FDF095E75EF94F908951
S12357C084E6891B809339068091A3079091A40792609093A4078093A30703C084E6809321
S12357E039068091BB049091BC048091CD0780911E0120910A0430910B0490E0C1968217B1
S123580093070CF489C0809100019091010181FF83C080910A0490910B04C397F4F0E091AB
S12358201C01F0911D0120911C0130911D0180910A0490910B0460911E0170E06E5C7F4FB4
S1235840AC01429FC001439F900D529F900D11240E942C30E61BF70B16C080910A0490919C
S12358600B04889764F480911C0190911D0196958795FC01EE0FFF1FE80FF91F04C0E0918E
S12358801C01F0911D018091BB049091BC0462E070E00E9440307093500660934F06CF0182
S12358A09695879590935206809351068091BB049091BC04E80FF91FF093BC04E093BB0483
S12358C08091BB049091BC0462E070E00E94403070935406609353068091180190E0909309
S12358E0560680935506309905C0809123019091240104C080911F01909120019093220154
S1235900809321018091A3079091A40782609093A4078093A30711C08091A3079091A40702
S12359208D7F9093A4078093A30780911F0190912001909322018093210180911406909192
S1235940150683FF1CC0E091BB04F091BC0420913D018091BB049091BC0464E170E00E9482
S1235960403030E0629FC001639F900D729F900D11248E0F9F1F9093BC048093BB0480913E
S123598000019091010190FF4DC08091F4039091F503823891050CF045C08091BB049091E0
S12359A0BC0420912A01820F911D9093BC048093BB04E091F403F091F503609118012091B7
S12359C02A0182E890E08E1B9F0B70E0AB01849FB001859F700D949F700D11248FEF90E027
S12359E0AB01489FB001499F700D589F700D1124882777FD8095982F30E040E050E00E9450
S1235A00013020E43FE140E050E00E945330C9012091BB043091BC04280F391F3093BC04EB
S1235A202093BB042091BB043091BC048091180145EF849FC00111248217930754F48091FC
S1235A401801849FC00111249093BC048093BB040BC08091BB049091BC041816190624F07E
S1235A601092BC041092BB048091BB049091BC0490936104809360048091600490916104B4
S1235A809093A7078093A60778941F910F9108951F920F920FB60F9211242F933F934F9315
S1235AA05F936F937F938F939F93AF93BF93EF93FF931092B100E091C304F0E02091A60727
S1235AC03091A70786B59091C504891B280F311DEE0FFF1FED5BF94F3183208386B58093B5
S1235AE013068091C304813019F40E94B3290AC08091C304823031F08091C304833011F074
S1235B008091C304FF91EF91BF91AF919F918F917F916F915F914F913F912F910F900FBEDD
S1235B200F901F9018951F93682F8FEF8093D1048091C5046093C50441E050E0162F181B58
S1235B40ACE0BEEF71E0FA01EE0FFF1FED5BF94F80819181181619066CF41093A507208161
S1235B6031818091A50790E080959095820F931F91838083FA01EE0FFF1FED5BF94F808107
S1235B8091811816190624F180819181855D9E4FFCF0413049F44093D00486B590E090939C
S1235BA05806809357060CC0423019F47093CC0707C0433019F47093D20402C070936106A6
S1235BC0FA01EE0FFF1FED5BF94FB183A08311C08091D104FA01EE0FFF1FED5BF94F2081C6
S1235BE0318190E02817390724F4808191818093D1044F5F5F4F4530510509F0A4CF809149
S1235C00D1048F3F21F08091D104860F87BD1F9108951F920F920FB60F9211242F933F933F
S1235C204F935F936F937F938F939F93AF93BF93EF93FF9386B50E94932DFF91EF91BF917F
S1235C40AF919F918F917F916F915F914F913F912F910F900FBE0F901F9018951F920F9287
S1235C600FB60F9211242F933F934F935F936F937F938F939F93AF93BF93EF93FF9386B5D2
S1235C800E94932DFF91EF91BF91AF919F918F917F916F915F914F913F912F910F900FBED2
S1235CA00F901F901895549A559A5C9A5D9A15BCEEE6F0E080818360808384E085BD16BC47
S1235CC082E187BD089511B88FEF84B915B887B98AB9089588E98093C1001092C50083E1FB
S1235CE08093C40087E598E09093150880931408909311088093100887E198E090931308F1
S1235D00809312089093980880939708109216081092420608951F920F920FB60F921124A9
S1235D208F939F93EF93FF9380911608882311F1E0911408F091150881918093C600F09382
S1235D401508E0931408E759F84030F087E598E09093150880931408809116088150809395
S1235D60160880911608882329F48091C1008F7D8093C100FF91EF919F918F910F900FBE8C
S1235D800F901F9018951F920F920FB60F9211242F938F939F93EF93FF938091C600E091A5
S1235DA09708F09198088083809142068F5F809342068091970890919808019690939808AF
S1235DC0809397088755984030F087E198E09093980880939708FF91EF919F918F912F91C4
S1235DE00F900FBE0F901F90189580914206882319F42FEF3FEF1AC0F8948091420681504B
S1235E0080934206E0911208F09113082191F0931308E0931208E755F84030F087E198E0AB
S1235E209093130880931208789430E0C9010895982F809116088F33E0F7809116088034FE
S1235E4010F080E00895F894809116088F5F80931608E0911008F091110890838091100808
S1235E6090911108019690931108809310088759984030F087E598E09093110880931008C3
S1235E808091C10080628093C100789481E00895CF93DF93EC0104C00E94182F81112196B5
S1235EA088818823C9F781E0DF91CF9108958EED93E00E94482F089586EE93E00E94482FF8
S1235EC008958091420608959F92AF92BF92CF92DF92EF92FF920F931F93DF93CF93CDB7D8
S1235EE0DEB729970FB6F894DEBF0FBECDBF7C01062FDE011196E9EEF3E089E001900D9287
S1235F008150E1F719E099E0A92EB12C6E010894C11CD11C8CE2982E002371F09501211B4F
S1235F203109802F90E02817390730F01150F601E10FF11D908200E01150F601E10FF11DC7
S1235F40C7016AE070E00E942C30805D8083C7016AE070E00E942C307B016115710511F430
S1235F60002311F00630C0F219E0141B7E010894E11CF11C07C0F701E10FF11D80810E9464
S1235F80182F1F5F1930B8F329960FB6F894DEBF0FBECDBFCF91DF911F910F91FF90EF9010
S1235FA0DF90CF90BF90AF909F900895DF92EF92FF920F931F937B018C01FB010995D82E35
S1235FC0C8010196F7010995982F8D2D1F910F91FF90EF90DF900895DF92EF92FF920F93B7
S1235FE01F93D72E7A018C01FA010995C80101966D2DF70109951F910F91FF90EF90DF90E8
S12360000895629FD001739FF001829FE00DF11D649FE00DF11D929FF00D839FF00D749F90
S1236020F00D659FF00D9927729FB00DE11DF91F639FB00DE11DF91FBD01CF011124089585
S1236040991B79E004C0991F961708F0961B881F7A95C9F780950895AA1BBB1B51E107C0A1
S1236060AA1FBB1FA617B70710F0A61BB70B881F991F5A95A9F780959095BC01CD0108952B
S123608097FB092E07260AD077FD04D0E5DF06D000201AF4709561957F4F0895F6F79095A4
S12360A081959F4F0895A1E21A2EAA1BBB1BFD010DC0AA1FBB1FEE1FFF1FA217B307E407DE
S12360C0F50720F0A21BB30BE40BF50B661F771F881F991F1A9469F760957095809590958A
S12360E09B01AC01BD01CF01089597FB092E05260ED057FD04D0D7DF0AD0001C38F4509571
S12361004095309521953F4F4F4F5F4F0895F6F790958095709561957F4F8F4F9F4F08955B
S1236120F894FFCF2F00010002000300040005000600070008003228E80390010614001EA0
S12361401E003C581B581B88136419121E01010203040A0411C4098813C4096400DCE640EE
S123616003020A1432469628000000000000000000000000000000000000000000000000C2
S12361800000000000000000000000000000000000000000000000000000000000000000FB
S12361A00000000000000000000102030405060708090A0B0C0D0E0F100102030405060737
S12361C008090A0B0C0D0E0F100102030405060708090A0B0C0D0E0F1014161718191A1B20
S12361E01C1D1E1F2021222324191A1B1C1D1E1F2021222324252627271E1F202223242589
S1236200262728292A2B2C2D2E000204060708090A0C0E28262422201E1E1E1E1E1E1E1E14
S12362201E1E1EF0FF80BBE0880465484BA438022BF0207019CC13860F440CC209D0074C1E
S1236240061B052A046A03D1025602F201A1015F012801FB00D600B7009D008700750066A9
S12362600059004D0044003C0034002E0029002500F0FF80BBE0880465484BA438022BF0BD
S1236280207019CC13860F440CC209D0074C061B052A046A03D1025602F201A1015F012896
S12362A001FB00D600B7009D0087007500660059004D0044003C0034002E0029002500F08C
S12362C0FF80BBE0880465484BA438022BF0207019CC13860F440CC209D0074C061B052A78
S12362E0046A03D1025602F201A1015F012801FB00D600B7009D0087007500660059004DB3
S12363000044003C0034002E0029002500F0FF80BBE0880465484BA438022BF0207019CC4D
S123632013860F440CC209D0074C061B052A046A03D1025602F201A1015F012801FB00D698
S123634000B7009D0087007500660059004D0044003C0034002E00290025000000F5047E36
S123636005AE066C08C00AB30D630F8B10D7118813000000000A000F001E003C007800FAED
S1236380007201E00180028002000008000A000C000E00C80A4A067E048403AC0D641A0013
S12363A02000270032003E0066008E00B202EB02240337034B03560361037003E800D600F0
S12363C0C200B0009D008A00780078006500520040002D00190007000000010001000117D2
S12363E05A5A5A505050505050505050505050500A0004010402030000030000FA3204042C
S119640004041B5B481B5B324A000D0A0020202020202020202093
S5030321D8
